:020000021000EC
:10E000004BC0000094C0000092C0000090C000000F
:10E010008EC000008CC000008AC0000088C00000D4
:10E0200086C0000084C00000C1C600007BC700009D
:10E030007EC000007CC000007AC0000078C00000F4
:10E0400076C0000074C0000072C0000070C0000004
:10E05000C2C000006CC000006AC0000068C00000C0
:10E0600066C0000064C0000062C0000060C0000024
:10E070005EC000005CC000005AC0000058C0000034
:10E0800056C0000054C0000052C0000050C0000044
:10E090004EC000004CC0000011241FBECFEFD0E2E4
:10E0A000DEBFCDBF85B7806890E00FB6F89485BF1E
:10E0B0000FBE85BF8C9A8FE19EE40197F1F700C0F7
:10E0C00000002FB1207185B790E08F770FB6F894DC
:10E0D00085BF0FBE85BF04B603FE0CC080918B02C6
:10E0E00090918C0282349C4D29F410928C021092F3
:10E0F0008B0202C0222319F0E0E0F0E0099512E063
:10E10000A0E0B1E0ECEFF4EF01E00BBF02C007903C
:10E110000D92A038B107D9F722E0A0E8B2E001C023
:10E120001D92AB38B207E1F709D00C947CFA68CFA6
:10E1300095B180959064892385B9089584B7877FC8
:10E1400084BF88E10FB6F89480936000109260005D
:10E150000FBE90E080E80FB6F89480936100909332
:10E1600061000FBEC1E0C5BF82E085BF269A2E9A2E
:10E1700002D6C0936F0083E08093810080E4D8DFF3
:10E18000789480910001882339F081E091E00E9429
:10E190004BF90E94D4F8F5CF8091800291E0980F5E
:10E1A000909380028F3F89F78091E0008160809397
:10E1B000E00082E49CED90938C0280938B022CE033
:10E1C00088E190E00FB6F894A895809360000FBEA8
:10E1D00020936000FFCF1F920F920FB60F92112471
:10E1E0008F9380E483B98F910F900FBE0F901F9093
:10E1F000189580E09DCF80E49BCF81E091E00E9464
:10E200002EF9882311F080E001C080E491CF81E0F5
:10E2100091E0E5C7CF93DF93EC0180E089DFCE0189
:10E22000CED0C82F80E084DF109280028C2FDF9147
:10E23000CF910895913039F0923051F080E090E024
:10E2400020E030E009C082E190E02CE032E004C040
:10E2500080E290E02CEE31E0FA01318320830895D2
:10E2600007B600FCFDCFF999FECF23E0FB018093B8
:10E270005B0020935700E89507B600FCFDCF81E1D5
:10E2800080935700E895089507B600FCFDCFF999F3
:10E29000FECF25E0FB0180935B0020935700E895BB
:10E2A00007B600FCFDCF81E180935700E895089503
:10E2B00007B600FCFDCFF999FECF21E00A01FB0172
:10E2C00080935B0020935700E8951124089521E284
:10E2D000FC01209357008491089529E0FC012093CC
:10E2E000570084910895E1E0F0E089E080935700C1
:10E2F0008491089507B600FCFDCFF999FECF809573
:10E3000099E0E1E0F0E0082E90935700E895089539
:10E310009F92AF92BF92CF92DF92EF92FF920F93B4
:10E320001F93CF93DF93EC01962EC8A0DF8CABA098
:10E33000BAA088E1C81681E0D80618F400E010E021
:10E3400015C080913C01807F856080933C0181E213
:10E35000809346011092470180E025C0C8018C0DD2
:10E360009D1D992039F005D20F5F1F4F0A151B051F
:10E37000A9F702C034D1F8CF6801E12CF12C89E073
:10E38000CC0CDD1CEE1CFF1C8A95D1F74C895D89F5
:10E390006E897F894C195D096E097F094C8B5D8BF5
:10E3A0006E8B7F8B81E0DF91CF911F910F91FF905A
:10E3B000EF90DF90CF90BF90AF909F900895EF9235
:10E3C000FF920F931F93CF93DF93EC018B8D8F31CF
:10E3D000A0F48D3108F0C0C08231F1F138F4882307
:10E3E00009F4BAC0833009F468C0BBC08A3109F4AB
:10E3F00091C08B3109F4A8C0B4C0883209F483C03D
:10E4000020F5853209F0ADC01092F1001092F100B4
:10E4100081E08093F10087E18093F1001092F10098
:10E420001092F10082E08093F1001092F10080914F
:10E43000E8008E778093E8004C895D896E897F893A
:10E4400048505109610971097AC08A3209F459C0EA
:10E450008F3209F481C085C00F8D1E8D8C8D837025
:10E4600019F48D8D882341F080913C01807F856077
:10E4700080933C0184E27CC078010532110518F0DC
:10E4800024E2E22EF12C40E050E0B7018EE192E070
:10E49000AAD260E070E0C8018E199F0967D280910E
:10E4A000E8008E778093E8004C895D896E897F89CA
:10E4B0004E195F096109710942C0EF8CFE2C82E19F
:10E4C0008E1510F492E1F92E0F2D10E040E050E08F
:10E4D000B8018AE391E087D28E2D90E060E070E091
:10E4E000801B910B43D28091E8008E778093E800E7
:10E4F0004C895D896E897F894F19510961097109BC
:10E500001EC060E001C061E0CE0102DF882309F493
:10E510003FC033C01092F1001092F1001092F10050
:10E520001092F1008091E8008E778093E8004C898A
:10E530005D896E897F8944505109610971094C8B4D
:10E540005D8B6E8B7F8B19C08F8D837091E08230D5
:10E5500009F490E0909300011C8A1D8A1E8A1F8A8C
:10E560000CC080913C01807F856080933C0180E2FB
:10E5700080934601109247010BC080913C01807F3F
:10E5800080933C01109246011092470181E001C046
:10E5900080E0DF91CF911F910F91FF90EF90089550
:10E5A000FB01F695E795E60FF0E0E80FF91F60FF35
:10E5B0000EC080818F70942F9295907F892B8083DD
:10E5C00084E0569547958A95E1F741830895408305
:10E5D000842F807F852B8183089574C77BC74F92DA
:10E5E0005F926F927F928F929F92AF92BF92CF92E3
:10E5F000DF92EF92FF920F931F93CF93DF93CDB7EC
:10E60000DEB7D2500FB6F894DEBF0FBECDBF8C017F
:10E6100040E050E060E072E0CE0101962BD28091A4
:10E62000E8008B778093E8000330110508F48AC076
:10E630000330110551F480EAFE013196ACE4B1E0FB
:10E6400001900D928A95E1F77DC08091A60190918D
:10E65000A7018150904C880F991F880F991F0817A8
:10E66000190778F48091E6019091E7018150904C70
:10E67000880F991F880F991F0817190708F044C0C1
:10E6800061C09C0121513F4F2017310758F36801A9
:10E69000C81AD90AE12CF12C79E0CC0CDD1CEE1C57
:10E6A000FF1C7A95D1F7CE0101965C014E019FEFD8
:10E6B000891A9DEF990AC11003C0C701B601D0DDC8
:10E6C000F501418150E0542F44278081482BC70138
:10E6D000B601EEDD26013701F2E04F0E511C611C40
:10E6E000711C411007C0C701B6016E5F7109810935
:10E6F0009109CADD82E0A80EB11CA814B90409F47E
:10E70000B1CF73016201D7CF9C01295F3F4F201722
:10E710003107C0F0081B190B102F0027110FFE0145
:10E7200031966F01E12CF12CF60161916F01C70167
:10E73000800F911F53DFFFEFEF1AFF0AE11482E011
:10E74000F80691F7DE5F0FB6F894DEBF0FBECDBFBF
:10E75000DF91CF911F910F91FF90EF90DF90CF90BD
:10E76000BF90AF909F908F907F906F905F904F90F1
:10E770000895AF92BF92CF92DF92EF92FF920F93E4
:10E780001F93CF93DF93CDB7DEB7C150D2400FB602
:10E79000F894DEBF0FBECDBF8E010F5F1F4F20E08C
:10E7A00032E0F801A901119241505040E1F7833065
:10E7B0009105B8F4019710F58EE3E2E4F2E0D80198
:10E7C00001900D928A95E1F785E5C150DE4F88836F
:10E7D000CF5FD1408AEAC050DE4F8883C050D2401C
:10E7E000A8C08330910509F044C080EAECE4F1E070
:10E7F000D80101900D928A95E1F79BC048EF5FE048
:10E8000060E070E0C801CCDE4FEF5FE061E070E0F7
:10E81000C801C6DE6091A6017091A70120E0CB017E
:10E8200001967C012B3311F0AC0102C04FEF5FE089
:10E83000C801CF5FDD4F2883C150D240B1DECF5F2A
:10E84000DD4F2881C150D2402F5FB7012C3339F7FB
:10E850006091E6017091E7017B019FEFE91AF90AE7
:10E86000A701C8019DDE4FEF5FE0B701C80198DE48
:10E8700060C02091A6013091A7012150304C220F99
:10E88000331F220F331F8217930770F42091E60184
:10E890003091E7012150304C220F331F220F331FDC
:10E8A0008217930740F545C0A90141515F4F4817B2
:10E8B000590760F3AC01421B530B60E070E0B9E014
:10E8C000440F551F661F771FBA95D1F7D8019E01D7
:10E8D0002F5F3D4F6A017B01EFEFCE1ADE0AEE0A91
:10E8E000FE0A6BBFFA0147914D93A217B30771F26D
:10E8F000B701A601EFCFA901495F5F4F481759073C
:10E90000C0F07C01E21AF30AFE2CEE24FF0C5E013B
:10E91000FFEFAF1AFDEFBF0A6801E01AF10AC70165
:10E920008C0D9D1D5ADEF60181936F01EA15FB05E2
:10E93000B1F740E050E060E072E0C80154D080914F
:10E94000E8008E778093E800CF5FDD4F0FB6F89434
:10E95000DEBF0FBECDBFDF91CF911F910F91FF9012
:10E96000EF90DF90CF90BF90AF900895EF92FF921D
:10E970000F931F93CF93DF938C01EB018DD1811106
:10E980002BC0209721F088819981081B190BE12C5D
:10E99000F12C01151105F9F08091E80085FD13C0F7
:10E9A0008091E8008E778093E800209741F088817D
:10E9B00099818E0D9F1D9983888385E00DC06CD150
:10E9C000882339F309C01092F100015011098FEF2B
:10E9D000E81AF80ADECF80E0DF91CF911F910F9106
:10E9E000FF90EF900895CF92DF92EF92FF920F93F6
:10E9F0001F93CF93DF937C018B01EA014DD18111ED
:10EA000030C0209731F088819981081B190BE80EDE
:10EA1000F91EC12CD12C0115110511F18091E800CE
:10EA200085FD13C08091E8008E778093E8002097E1
:10EA300041F0888199818C0D9D1D9983888385E0A3
:10EA400010C02AD1882339F30CC0F70181917F01CE
:10EA50008093F10001501109FFEFCF1ADF0ADBCFDD
:10EA600080E0DF91CF911F910F91FF90EF90DF90A9
:10EA7000CF900895CF92DF92EF92FF920F931F9362
:10EA8000CF93DF937C018B01EA0106D1811130C065
:10EA9000209731F088819981081B190BE80EF91E27
:10EAA000C12CD12C0115110511F18091E80085FDD3
:10EAB00013C08091E8008B778093E800209741F0A5
:10EAC000888199818C0D9D1D9983888385E010C074
:10EAD000E3D0882339F30CC08091F100F7018193D2
:10EAE0007F0101501109FFEFCF1ADF0ADBCF80E071
:10EAF000DF91CF911F910F91FF90EF90DF90CF901A
:10EB000008952091890230918A022617370748F02C
:10EB10006115710539F42091E8002E772093E80003
:10EB200001C0B901FC0120E06115710591F18EB3BE
:10EB30008823E1F18530E1F18091E80083FD3AC05E
:10EB40008091E80082FF06C08091E80082FF24C027
:10EB500080E008958091E80080FFE6CF8091F20088
:10EB60009091F3006115710551F08830910538F4EA
:10EB700021912093F100615071090196F3CF21E0BA
:10EB8000089709F020E08091E8008E778093E800F4
:10EB9000CBCF2111CCCFD8CF8EB3882339F085309D
:10EBA00039F08091E80083FFCFCF04C082E0089560
:10EBB00083E0089581E008958F708093E900EBEE83
:10EBC000F0E0808181608083EDEEF0E01082609360
:10EBD000EC0040838091EE00881F8827881F0895ED
:10EBE0000F931F93CF93DF93062FEC0110E01017C4
:10EBF00071F19881992341F12C81E981FA817B811E
:10EC0000892F8F70873010F080E022C0223010F002
:10EC100056E001C052E028E030E040E02E173F0708
:10EC200020F44F5F220F331FF9CF4295407F452BD1
:10EC3000692F661F6627661F90E4799F9001112453
:10EC4000622BBADF882301F31F5F2596D0CF81E0C6
:10EC5000DF91CF911F910F9108958091830287FDDD
:10EC600005C08091E80080FF0DC010C08091E800D1
:10EC700082FD04C08EB38111F9CF08958091E80020
:10EC80008B7707C08EB38111ECCF08958091E80097
:10EC90008E778093E80008958091E4009091E500DC
:10ECA00045E62091EC0020FF20C02091E80020FDE7
:10ECB00020C02EB3222389F0253089F02091EB006B
:10ECC00025FD0FC02091E4003091E5002817390799
:10ECD00041F3415041F0C901E4CF82E0089583E05F
:10ECE000089581E0089584E008952091E80022FFCE
:10ECF000E0CF80E008950F931F93CF93DF9349D027
:10ED000050D0C8EDD0E088818F7788838881806873
:10ED1000888388818F7D8883E7EDF0E0808180683B
:10ED2000808319BC1EBA1092810200EE10E0F80137
:10ED300080818B7F808388818160888342E060E06E
:10ED400080E03ADFE1EEF0E080818E7F8083E2EECA
:10ED5000F0E0808181608083808188608083F80119
:10ED600080818E7F8083888180618883DF91CF91CD
:10ED70001F910F910895E8EDF0E080818F7E8083F0
:10ED8000E7EDF0E080818160808381E08093820202
:10ED9000B2CFE8EDF0E080818C7F80831092E200BA
:10EDA00008951092DA001092E10008951F920F92D8
:10EDB0000FB60F9211240BB60F922F933F934F93E0
:10EDC0005F936F937F938F939F93AF93BF93EF93D3
:10EDD000FF938091DA0080FF1BC08091D80080FFF4
:10EDE00017C08091DA008E7F8093DA008091D9007D
:10EDF00080FF0BC08CE089BD8EE089BD09B400FEA8
:10EE0000FDCF81E08EBBF5D903C019BC1EBAF3D982
:10EE10008091E10080FF17C08091E20080FF13C065
:10EE20008091E2008E7F8093E2008091E200806119
:10EE30008093E2008091D80080628093D80019BC52
:10EE400085E08EBBB0D18091E10084FF2EC080911F
:10EE5000E20084FF2AC08CE089BD8EE089BD09B440
:10EE600000FEFDCF8091D8008F7D8093D8008091E7
:10EE7000E1008F7E8093E1008091E2008F7E80939D
:10EE8000E2008091E20081608093E2008091810243
:10EE9000882311F084E007C08091E30087FF02C05F
:10EEA00083E001C081E08EBB7ED18091E10083FFD1
:10EEB00026C08091E20083FF22C08091E100877F1D
:10EEC0008093E10082E08EBB109281028091E1008C
:10EED0008E7F8093E1008091E2008E7F8093E2003C
:10EEE0008091E20080618093E20042E060E080E097
:10EEF00063DE8091F00088608093F00054D1FF9130
:10EF0000EF91BF91AF919F918F917F916F915F91A1
:10EF10004F913F912F910F900BBE0F900FBE0F900E
:10EF20001F9018951F920F920FB60F9211240BB6D7
:10EF30000F922F933F934F935F936F937F938F9392
:10EF40009F93AF93BF93CF93EF93FF93C091E9004B
:10EF5000CF708091EC001092E9008091F000877FE3
:10EF60008093F00078941DD01092E9008091F00019
:10EF700088608093F000C093E900FF91EF91CF91FA
:10EF8000BF91AF919F918F917F916F915F914F91C1
:10EF90003F912F910F900BBE0F900FBE0F901F90BF
:10EFA00018951F93CF93DF9300D0CDB7DEB7E3E87A
:10EFB000F2E08091F100819382E0EB38F807C9F725
:10EFC00026D98091E80083FFDAC090918302809176
:10EFD0008402853009F465C030F4813059F168F05D
:10EFE000833041F1CCC0883009F49CC0893009F4E9
:10EFF000ABC0863009F0C3C075C0903881F092383C
:10F0000009F0BDC0809187028F708093E9009091D4
:10F01000EB0095FB992790F91092E90001C090E070
:10F020008091E800877F8093E8009093F100109230
:10F03000F10083C0292F2D7F09F0A1C0923009F083
:10F040009EC090918502911126C0209187022F7059
:10F0500009F495C02093E9009091EB0090FF1BC04C
:10F06000833021F48091EB00806213C08091EB002B
:10F0700080618093EB0081E090E0022E01C0880F58
:10F080000A94EAF78093EA001092EA008091EB007C
:10F0900088608093EB001092E9008091E800877F00
:10F0A0004FC091116CC0109185021F778091E300D1
:10F0B0008078812B8093E3008091E800877F8093A4
:10F0C000E800CBDD8091E80080FFFCCF8091E30079
:10F0D00080688093E300112311F083E001C082E097
:10F0E0008EBB4DC09058923008F049C0AE014F5FC2
:10F0F0005F4F6091870280918502909186029AD835
:10F10000009709F43CC02091E800277F2093E80095
:10F11000BC0189819A81F5DC8091E8008B7780932E
:10F12000E8002DC0903859F58091E800877F8093E2
:10F13000E800809181028093F1008091E8008E7751
:10F140008093E8008ADD1BC0911119C0909185025F
:10F150009230A8F48091E800877F8093E800909334
:10F1600081027BDD80918102811104C08091E300E6
:10F1700087FF02C084E001C081E08EBB3ED8809151
:10F18000E80083FF0AC08091E800877F8093E80051
:10F190008091EB0080628093EB000F900F90DF91E5
:10F1A000CF911F9108950895CF938EB38823A9F02E
:10F1B0008091E9008F709091EC0090FF02C090E880
:10F1C00001C090E0C92FC82B1092E9008091E8009F
:10F1D00083FDE7DECF70C093E900CF910895CF9310
:10F1E000DF93EC018091E80083FF35C0888190E0D7
:10F1F00020918702309188022817390761F58091A4
:10F2000084028E3F79F08F3F31F580918302813205
:10F2100011F58091E800877F8093E8001EDD81E092
:10F2200088AF19C080918302813AA9F48091E800E7
:10F23000877F8093E8008091E80080FFFCCF8B857A
:10F2400081508093F1008091E8008E778093E800F0
:10F25000DF91CF9102CDDF91CF910895CF93DF93CE
:10F26000EC01FC013C968DE2DF011D928A95E9F7E5
:10F2700082E08C83898761E0CE010196B1DC88232E
:10F2800031F061E0CE010696DF91CF91A9CC80E00C
:10F29000DF91CF910895EF92FF920F931F93CF9339
:10F2A000DF9300D0CDB7DEB78C018EB3843009F088
:10F2B00000C1F80186818F708093E9008091E80099
:10F2C00082FFBDC086818F708093E9001A82198207
:10F2D0007801FCE0EF0EF11CAE014F5F5F4F6FE075
:10F2E00070E0C701C7DBF801853021F480AD8823C9
:10F2F00099F3A5C084859585A685B7858535934501
:10F30000A244B34461F4F801918D8385981738F4D1
:10F31000808D8F7121F4828D8150803180F08091B9
:10F32000EB0080628093EB00F80181818F70809305
:10F33000E9008091EB0080628093EB0080C01A822C
:10F3400019827801FBE1EF0EF11CF801628D70E08B
:10F35000AE014F5F5F4FC7018DDB853029F4F801A7
:10F3600080AD882391F36BC08091E8008B77809308
:10F37000E800F801808D87FF04C081818F70809341
:10F38000E900C8010E940AF191E09827F80197ABC3
:10F3900045E553E562E473E543A754A765A776A75F
:10F3A000408951896289738947A750AB61AB72ABC1
:10F3B000448955896689778943AB54AB65AB76AB95
:10F3C000811109C0452B462B472B29F08091EB007A
:10F3D00080628093EB00F80186818F708093E90052
:10F3E0008091EB00F80185FF04C080AD8823C1F354
:10F3F00026C081818F708093E9008091EB0085FFAA
:10F4000005C0F80180AD8823C1F319C01A821982A2
:10F410007801FBE2EF0EF11CAE014F5F5F4F6DE034
:10F4200070E0C701E0DA853029F4F80180AD882367
:10F4300099F305C08091E8008E778093E800F80189
:10F4400080AD8823B1F126812F7081E090E0AC017E
:10F4500002C0440F551F2A95E2F74093EA0010922C
:10F46000EA0021812F70022E01C0880F0A94EAF76A
:10F470008093EA001092EA0086818F708093E90001
:10F480008091EB0080618093EB008091EB008860BD
:10F490008093EB0081818F708093E9008091EB0075
:10F4A00080618093EB008091EB0088608093EB009B
:10F4B00010AE0F900F90DF91CF911F910F91FF90A1
:10F4C000EF900895F999FECF92BD81BDF89A9927E2
:10F4D00080B50895262FF999FECF92BD81BDF89A87
:10F4E000019700B4021639F01FBA20BD0FB6F89488
:0CF4F000FA9AF99A0FBE0895F894FFCF25
:10F4FC0001008340000001044000000101000000F5
:10F50C0000000000000000000000000000000000EF
:10F51C0000000000000000000000000000000000DF
:10F52C00000000000000000000007000000000005F
:10F53C00000A000000000000000000004C5546418D
:10F54C0020424F4F54202008000000000000000013
:10F55C000000000000000000000000004146004CCC
:10F56C00004100530048000F00262E0042004900C5
:10F57C004E0000000000000000000000464C41530B
:10F58C004820202042494E000000000000000000EE
:10F59C00000020084E12020000E001004145004529
:10F5AC0000500052004F000F00144D002E0042007E
:10F5BC0049004E000000000000000000454550527C
:10F5CC004F4D202042494E0000000000000000007A
:10F5DC00000020084E123E00FF0F00000902200020
:10F5EC0001010080320904000002080650000705E2
:10F5FC0083024000050705040240000512011001BA
:10F60C0000000008EB034520010000000001008011
:10F61C0000021F0000004C55464100000000426FE4
:10F62C006F746C6F61646572000000000000302E16
:10F63C003030EB3C906D6B646F73667300000204AA
:10F64C0001000210001801F801001800040000006D
:10F65C00000000000000000029785634124C55467A
:10F66C004120424F4F54202046415431322020201B
:10FFA0000C9430F10C9444F10C9458F10C9467F1DA
:10FFB0000C946DF10C9473F10C947AF108950895FA
:06FFC00008950895089564
:10FFE000DFCFE0CFE1CFE2CFE3CFE4CFE5CFE6CF85
:08FFF000E6CFE6CFE6CFE6CF35
:08FFF80000E0010030DFFBDC3A
:040000031000E00009
:00000001FF
